:020000040000FA
:04080000F1EF04F020
:1008100003B23DEF04F0F2B458EF04F09EB060EF85
:1008200004F09EB268EF04F0F2A81AEF04F0F2B2FE
:100830001CEF04F0CFEF04F0CD90F29207BC078ECE
:10084000078C9EA029EF04F00101463F29EF04F038
:10085000472B07AE34EF04F0CECF51F1CFCF52F19A
:1008600046C153F147C154F1CF6ACE6A0101466BCC
:10087000476B9E90CD80CFEF04F00392030103EE0F
:1008800000F080517F0BE92604C0EFFF802B8151DF
:10089000805D700BD8A48B8200008051815D700B4D
:1008A000D8A48B9281518019D8B40790CFEF04F06F
:1008B000F2940101383FCFEF04F0392BCFEF04F071
:1008C0009E900101463FCFEF04F0472BCFEF04F09D
:1008D0009E92C3CF48F1C4CF49F1C28207B492EFD0
:1008E00004F03AC13EF13BC13FF13CC140F13DC192
:1008F00041F151C155F152C156F153C157F154C1A3
:1009000058F1010148514E2749514F23E86A5023BD
:100910000D2E92EF04F04FC14AF150C14BF14E6BD6
:100920004F6B506B0201002FCFEF04F03C0E006FB5
:10093000D57ED5BE32D0D6CF3AF1D7CF3BF138C134
:100940003CF1E86AE8CF3DF1010147A7B3EF04F0BD
:10095000079C079E0101000E516F600E526F3D0E05
:10096000536F080E546F01013ABFC3EF04F03B67A9
:10097000C3EF04F03C67C3EF04F03D67C3EF04F03E
:10098000F288C8EF04F0F298516B526B536B546BC2
:10099000D76AD66A0101386B396BCFEF04F002C019
:1009A000E0FF005001C0D8FF1000A6B2D5EF04F060
:1009B0000CC0A9FF0BC0A8FFA69EA69CA684F29E11
:1009C000550EA76EAA0EA76EA682F28EA694A6B2A8
:1009D000E7EF04F01200A96EA69EA69CA680A85080
:1009E0001200076A0F010E0EC16E860EC06E030E56
:1009F000C26E0F01896A110E926E080E8A6EF10E98
:100A0000936E8B6A800E946EF18E0D6A4E6B4F6BF7
:100A1000506B4A6B4B6B0F01280ED56EF28AB00EED
:100A2000CD6E9D800101516B526B536B546B556BB6
:100A3000566B576B586B596B5A6B5B6B5C6B079CB7
:100A4000079E760ECA6E9D8202013C0E006FCC6A34
:100A5000240EAC6E0401806B816B0F01900EAB6EA7
:100A60000F019D8A0301806B816BA26B8B920790B3
:100A70000001F28EF28C07B099EF0CF08B74030139
:100A8000805181197F0BD8B499EF0CF013EE00F070
:100A900081517F0BE126812BE7CFE8FFE00BD8B433
:100AA00099EF0CF023EE82F0A2511F0BD926E7CF6D
:100AB000DFFFA22BDF50780AD8A499EF0CF0078053
:100AC0008251720AD8B41BEF07F08251630AD8B47E
:100AD00059EF09F08251690AD8B48EEF05F08251BE
:100AE0007A0AD8B4A1EF06F08EEF09F0040114EEF3
:100AF00000F080517F0BE12682C4E7FF802B1200BB
:100B00000D0E826F76EC05F00A0E826F76EC05F022
:100B10001200040E826F76EC05F012000401690EDB
:100B2000826F76EC05F004012C0E826F76EC05F0F6
:100B30000101030E006F000E016F000E026F000E28
:100B4000036F28EC0FF020C182F40401300E8227DD
:100B500076EC05F021C182F40401300E822776EC98
:100B600005F022C182F40401300E822776EC05F0F4
:100B700023C182F40401300E822776EC05F024C1F3
:100B800082F40401300E822776EC05F025C182F450
:100B90000401300E822776EC05F026C182F40401B0
:100BA000300E822776EC05F027C182F40401300E66
:100BB000822776EC05F004012C0E826F76EC05F0AE
:100BC0000101030E006F000E016F000E026F000E98
:100BD000036F28EC0FF020C182F40401300E82274D
:100BE00076EC05F021C182F40401300E822776EC08
:100BF00005F022C182F40401300E822776EC05F064
:100C000023C182F40401300E822776EC05F024C162
:100C100082F40401300E822776EC05F025C182F4BF
:100C20000401300E822776EC05F026C182F404011F
:100C3000300E822776EC05F027C182F40401300ED5
:100C4000822776EC05F004012C0E826F76EC05F01D
:100C500001010C0E006F000E016F000E026F000EFE
:100C6000036F28EC0FF020C182F40401300E8227BC
:100C700076EC05F021C182F40401300E822776EC77
:100C800005F022C182F40401300E822776EC05F0D3
:100C900023C182F40401300E822776EC05F024C1D2
:100CA00082F40401300E822776EC05F025C182F42F
:100CB0000401300E822776EC05F026C182F404018F
:100CC000300E822776EC05F027C182F40401300E45
:100CD000822776EC05F004012C0E826F76EC05F08D
:100CE000200EF86EF76AF66A04010900F5CF82F467
:100CF00076EC05F00900F5CF82F476EC05F00900FA
:100D0000F5CF82F476EC05F00900F5CF82F476ECAD
:100D100005F00900F5CF82F476EC05F00900F5CF77
:100D200082F476EC05F00900F5CF82F476EC05F05C
:100D30000900F5CF82F476EC05F080EC05F08EEF3B
:100D400009F08351630AD8A48EEF09F08451610A37
:100D5000D8A48EEF09F085516C0AD8A48EEF09F063
:100D60008651410A42E08651440A1BE08651420AFC
:100D7000D8B408EF07F08651350AD8B417EF0BF056
:100D80008651360AD8B46BEF0BF08651370AD8B4C7
:100D9000D3EF0BF08651380AD8B431EF0CF08EEF58
:100DA00009F00798079A04017A0E826F76EC05F035
:100DB0000401780E826F76EC05F00401640E826FF8
:100DC00076EC05F081A8ECEF06F00401550E826F79
:100DD00076EC05F0F1EF06F004014C0E826F76EC34
:100DE00005F080EC05F08EEF09F00788079A040102
:100DF0007A0E826F76EC05F00401410E826F76EC7C
:100E000005F00401610E826F76EC05F0E2EF06F06A
:100E10000798078A04017A0E826F76EC05F00401C8
:100E2000420E826F76EC05F00401610E826F76EC63
:100E300005F0E2EF06F00401720E826F76EC05F029
:100E400004012C0E826F76EC05F0078455C159F130
:100E500056C15AF157C15BF158C15CF13EC142F134
:100E60003FC143F140C144F141C145F14AC14CF198
:100E70004BC14DF107940101620E046F010E056F25
:100E8000000E066F000E076F59C100F15AC101F143
:100E90005BC102F15CC103F18EEC0EF003BF98EF71
:100EA00007F00E0EEBEC04F0E8CF0CF10F0EEBECBC
:100EB00004F0E8CF0DF1100EEBEC04F0E8CF0EF1EA
:100EC000110EEBEC04F0E8CF0FF1D7EC0DF059C1A7
:100ED00004F15AC105F15BC106F15CC107F18EEC6A
:100EE0000EF007829BEC0DF0D7EC0DF007929BEC17
:100EF0000DF059C100F15AC101F15BC102F15CC1B1
:100F000003F107929BEC0DF0CC0E046FE00E056F21
:100F1000870E066F050E076F8EEC0EF000C10CF108
:100F200001C10DF102C10EF103C10FF1D1EF07F0C4
:100F30000101800E006F1A0E016F060E026F000E87
:100F4000036F42C104F143C105F144C106F145C13B
:100F500007F18EEC0EF003AFB2EF07F085EC0FF067
:100F6000E4EF07F00E0EEBEC04F0E8CF0CF10F0EFF
:100F7000EBEC04F0E8CF0DF1100EEBEC04F0E8CF51
:100F80000EF1110EEBEC04F0E8CF0FF142C100F1CD
:100F900043C101F144C102F145C103F107829BEC59
:100FA0000DF00CC100F10DC101F10EC102F10FC134
:100FB00003F10101000E046F000E056F010E066FB4
:100FC000000E076FBCEC0EF028EC0FF01D67EEEF83
:100FD00007F00401200E826FF1EF07F004012D0EDF
:100FE000826F76EC05F024C182F40401300E822772
:100FF00076EC05F025C182F40401300E822776ECF0
:1010000005F004012E0E826F76EC05F026C182F405
:101010000401300E822776EC05F027C182F404012A
:10102000300E822776EC05F004016D0E826F76ECAF
:1010300005F004012C0E826F76EC05F042C100F140
:1010400043C101F144C102F145C103F1010128ECA2
:101050000FF01EC182F40401300E822776EC05F0F9
:101060001FC182F40401300E822776EC05F020C106
:1010700082F40401300E822776EC05F021C182F45F
:101080000401300E822776EC05F022C182F40401BF
:10109000300E822776EC05F023C182F40401300E75
:1010A000822776EC05F024C182F40401300E8227F9
:1010B00076EC05F025C182F40401300E822776EC2F
:1010C00005F026C182F40401300E822776EC05F08B
:1010D00027C182F40401300E822776EC05F004016A
:1010E000480E826F76EC05F004017A0E826F76EC82
:1010F00005F004012C0E826F76EC05F059C100F169
:101100005AC101F15BC102F15CC103F1010128EC9C
:101110000FF01EC182F40401300E822776EC05F038
:101120001FC182F40401300E822776EC05F020C145
:1011300082F40401300E822776EC05F021C182F49E
:101140000401300E822776EC05F022C182F40401FE
:10115000300E822776EC05F023C182F40401300EB4
:10116000822776EC05F024C182F40401300E822738
:1011700076EC05F025C182F40401300E822776EC6E
:1011800005F026C182F40401300E822776EC05F0CA
:1011900027C182F40401300E822776EC05F00401A9
:1011A000630E826F76EC05F004012C0E826F76ECF4
:1011B00005F059C100F15AC101F15BC102F15CC1F6
:1011C00003F101010A0E046F000E056F000E066F99
:1011D000000E076F9DEC0EF0000E046F120E056FEF
:1011E000000E066F000E076FBCEC0EF028EC0FF03F
:1011F0001EC182F40401300E822776EC05F01FC177
:1012000082F40401300E822776EC05F020C182F4CE
:101210000401300E822776EC05F021C182F404012E
:10122000300E822776EC05F022C182F40401300EE4
:10123000822776EC05F023C182F40401300E822768
:1012400076EC05F024C182F40401300E822776EC9E
:1012500005F004012E0E826F76EC05F025C182F4B4
:101260000401300E822776EC05F026C182F40401D9
:10127000300E822776EC05F027C182F40401300E8F
:10128000822776EC05F00401730E826F76EC05F090
:1012900004012C0E826F76EC05F085EC0FF04CC14A
:1012A00000F14DC101F1B7EC0AF080EC05F08EEFD2
:1012B00009F00401630E826F76EC05F004012C0E38
:1012C000826F76EC05F093EC09F004012C0E826F2E
:1012D00076EC05F006EC0AF004012C0E826F76EC39
:1012E00005F082EC0AF004012C0E826F76EC05F01A
:1012F0000101F80E006FCD0E016F660E026F030E36
:10130000036FA8EC09F004012C0E826F76EC05F057
:1013100098EC0AF080EC05F08EEF09F00301A26B67
:10132000079099EF0CF0D8900E0EEBEC04F0E8CF9C
:1013300000F10F0EEBEC04F0E8CF01F1100EEBEC36
:1013400004F0E8CF02F1110EEBEC04F0E8CF03F16A
:101350000101000E046F000E056F010E066F000EF6
:10136000076FBCEC0EF028EC0FF01EC182F40401F4
:10137000300E822776EC05F01FC182F40401300E96
:10138000822776EC05F020C182F40401300E82271A
:1013900076EC05F021C182F40401300E822776EC50
:1013A00005F022C182F40401300E822776EC05F0AC
:1013B00023C182F40401300E822776EC05F024C1AB
:1013C00082F40401300E822776EC05F025C182F408
:1013D0000401300E822776EC05F004012E0E826F98
:1013E00076EC05F026C182F40401300E822776ECFB
:1013F00005F027C182F40401300E822776EC05F057
:1014000004016D0E826F76EC05F01200120EEBEC0B
:1014100004F0E8CF00F1130EEBEC04F0E8CF01F19B
:10142000140EEBEC04F0E8CF02F1150EEBEC04F037
:10143000E8CF03F101010A0E046F000E056F000EE4
:10144000066F000E076F9DEC0EF0000E046F120E7B
:10145000056F000E066F000E076FBCEC0EF028EC57
:101460000FF01EC182F40401300E822776EC05F0E5
:101470001FC182F40401300E822776EC05F020C1F2
:1014800082F40401300E822776EC05F021C182F44B
:101490000401300E822776EC05F022C182F40401AB
:1014A000300E822776EC05F023C182F40401300E61
:1014B000822776EC05F024C182F40401300E8227E5
:1014C00076EC05F004012E0E826F76EC05F025C156
:1014D00082F40401300E822776EC05F026C182F4F6
:1014E0000401300E822776EC05F027C182F4040156
:1014F000300E822776EC05F00401730E826F76ECD5
:1015000005F012000A0EEBEC04F0E8CF00F10B0E30
:10151000EBEC04F0E8CF01F10C0EEBEC04F0E8CFBB
:1015200002F10D0EEBEC04F0E8CF03F1B7EF0AF097
:10153000060EEBEC04F0E8CF00F1070EEBEC04F044
:10154000E8CF01F1080EEBEC04F0E8CF02F1090E50
:10155000EBEC04F0E8CF03F1B7EF0AF0010185EC02
:101560000FF007844AC100F14BC101F1079401015A
:10157000E80E046F800E056F000E066F000E076FF9
:101580009DEC0EF0000E046F040E056F000E066F4A
:10159000000E076FBCEC0EF0880E046F130E056F83
:1015A000000E066F000E076F8EEC0EF00A0E046F31
:1015B000000E056F000E066F000E076FBCEC0EF0FC
:1015C00028EC0FF001011D67EBEF0AF00401200E7B
:1015D000826FEEEF0AF004012D0E826F76EC05F0BB
:1015E00024C182F40401300E822776EC05F025C177
:1015F00082F40401300E822776EC05F026C182F4D5
:101600000401300E822776EC05F004012E0E826F65
:1016100076EC05F027C182F40401300E822776ECC7
:1016200005F00401430E826F76EC05F0120087C3CB
:101630001EF188C31FF189C320F18AC321F18BC336
:1016400022F18CC323F18DC324F18EC325F190C305
:1016500026F191C327F10101D2EC0FF04AEC0FF013
:101660000101000E046F000E056F010E066F000EE3
:10167000076F9DEC0EF00E0E0C6E00C10BF0D5EC5A
:1016800004F00F0E0C6E01C10BF0D5EC04F0100E3F
:101690000C6E02C10BF0D5EC04F0110E0C6E03C100
:1016A0000BF0D5EC04F004017A0E826F76EC05F0B5
:1016B00004012C0E826F76EC05F00401350E826F6A
:1016C00076EC05F004012C0E826F76EC05F093ECBD
:1016D00009F0F1EF06F087C31EF188C31FF189C33B
:1016E00020F18AC321F18BC322F18CC323F18DC376
:1016F00024F18EC325F190C326F191C327F1010196
:10170000D2EC0FF04AEC0FF0880E046F130E056F49
:10171000000E066F000E076F92EC0EF0000E046FC5
:10172000040E056F000E066F000E076F9DEC0EF0A5
:101730000101E80E046F800E056F000E066F000EAB
:10174000076FBCEC0EF00A0E0C6E00C10BF0D5EC6E
:1017500004F00B0E0C6E01C10BF0D5EC04F00C0E76
:101760000C6E02C10BF0D5EC04F00D0E0C6E03C133
:101770000BF0D5EC04F004017A0E826F76EC05F0E4
:1017800004012C0E826F76EC05F00401360E826F98
:1017900076EC05F004012C0E826F76EC05F082ECFD
:1017A0000AF0F1EF06F087C31EF188C31FF189C369
:1017B00020F18AC321F18BC322F18CC323F18DC3A5
:1017C00024F18FC325F190C326F191C327F10101C4
:1017D000D2EC0FF04AEC0FF0000E046F120E056F02
:1017E000000E066F000E076F9DEC0EF001010A0E51
:1017F000046F000E056F000E066F000E076FBCEC45
:101800000EF0120E0C6E00C10BF0D5EC04F0130EAE
:101810000C6E01C10BF0D5EC04F0140E0C6E02C17D
:101820000BF0D5EC04F0150E0C6E03C10BF0D5ECEB
:1018300004F004017A0E826F76EC05F004012C0EA0
:10184000826F76EC05F00401370E826F76EC05F0BE
:1018500004012C0E826F76EC05F006EC0AF0F1EF35
:1018600006F087C31EF188C31FF189C320F18AC324
:1018700021F18BC322F18CC323F18DC324F18EC3DC
:1018800025F190C326F191C327F10101D2EC0FF0AD
:101890004AEC0FF0880E046F130E056F000E066FF2
:1018A000000E076F92EC0EF0000E046F040E056F31
:1018B000000E066F000E076F9DEC0EF00101E80EA2
:1018C000046F800E056F000E066F000E076FBCECF4
:1018D0000EF0060E0C6E00C10BF0D5EC04F0070EF6
:1018E0000C6E01C10BF0D5EC04F0080E0C6E02C1B9
:1018F0000BF0D5EC04F0090E0C6E03C10BF0D5EC27
:1019000004F004017A0E826F76EC05F004012C0ECF
:10191000826F76EC05F00401380E826F76EC05F0EC
:1019200004012C0E826F76EC05F098EC0AF0F1EFD2
:1019300006F081A857EF0DF007A810EF0DF0010198
:10194000800E006F1A0E016F060E026F000E036FFD
:101950003EC104F13FC105F140C106F141C107F1AB
:101960008EEC0EF003BF57EF0DF095EC0DF03EC17D
:1019700000F13FC101F140C102F141C103F1078211
:101980009BEC0DF00CC104F10DC105F10EC106F187
:101990000FC107F1F80E006FCD0E016F660E026FDA
:1019A000030E036F8EEC0EF00E0E0C6E00C10BF0EA
:1019B000D5EC04F00F0E0C6E01C10BF0D5EC04F069
:1019C000100E0C6E02C10BF0D5EC04F0110E0C6E73
:1019D00003C10BF0D5EC04F00784010185EC0FF096
:1019E0004AC100F14BC101F107940A0E0C6E00C10F
:1019F0000BF0D5EC04F00B0E0C6E01C10BF0D5EC26
:101A000004F00C0E0C6E02C10BF0D5EC04F00D0EC0
:101A10000C6E03C10BF0D5EC04F0079857EF0DF0F6
:101A200007AA57EF0DF00784010185EC0FF04AC1BA
:101A300000F14BC101F10794060E0C6E00C10BF0D2
:101A4000D5EC04F0070E0C6E01C10BF0D5EC04F0E0
:101A5000080E0C6E02C10BF0D5EC04F0090E0C6EF2
:101A600003C10BF0D5EC04F0078455C100F156C159
:101A700001F157C102F158C103F10794120E0C6E27
:101A800000C10BF0D5EC04F0130E0C6E01C10BF08D
:101A9000D5EC04F0140E0C6E02C10BF0D5EC04F082
:101AA000150E0C6E03C10BF0D5EC04F0079A04017F
:101AB000805181197F0B0BE09EA809D014EE00F035
:101AC00081517F0BE126E750812B0F01AD6E3BEF7B
:101AD00005F00CC100F10DC101F10EC102F10FC101
:101AE00003F1000E046F000E056F010E066F000E6D
:101AF000076FBCEC0EF01DA194EF0DF01451D8B49B
:101B000094EF0DF00CC100F10DC101F10EC102F115
:101B10000FC103F1000E046F000E056F0A0E066F71
:101B2000000E076FBCEC0EF0120001010C6B0D6B88
:101B30000E6B0F6B12000101005305E1015303E12D
:101B4000025301E1002B5EEC0EF085EC0FF02C51FE
:101B5000006F2D51016F420E046F4B0E056F000E8A
:101B6000066F000E076F9DEC0EF000C104F101C17D
:101B700005F102C106F103C107F10CC100F10DC16D
:101B800001F10EC102F10FC103F107B2CCEF0DF06C
:101B900092EC0EF0CEEF0DF08EEC0EF000C10CF1D9
:101BA00001C10DF102C10EF103C10FF1120085EC6C
:101BB0000FF04CC100F14DC101F1060EEBEC04F049
:101BC000E8CF04F1070EEBEC04F0E8CF05F1080EC6
:101BD000EBEC04F0E8CF06F1090EEBEC04F0E8CFF3
:101BE00007F18EEC0EF000C118F101C119F102C12C
:101BF0001AF103C11BF1290E046F000E056F000ED0
:101C0000066F000E076F9DEC0EF0EE0E046F430E94
:101C1000056F000E066F000E076F92EC0EF018C1F4
:101C200004F119C105F11AC106F11BC107F19DECC0
:101C30000EF000C110F101C111F102C112F103C196
:101C400013F1120EEBEC04F0E8CF04F1130EEBEC01
:101C500004F0E8CF05F1140EEBEC04F0E8CF06F148
:101C6000150EEBEC04F0E8CF07F10D0E006F000E3F
:101C7000016F000E026F000E036F9DEC0EF0180E48
:101C8000046F000E056F000E066F000E076FBCECB0
:101C90000EF010C104F111C105F112C106F113C11A
:101CA00007F192EC0EF06A0E046F2A0E056F000E1B
:101CB000066F000E076F8EEC0EF01200BF0EFA6E6C
:101CC000200E2D6F2C6BD890003701370237033769
:101CD000D8B06FEF0EF02D2F64EF0EF02C072D070C
:101CE0000353D8B412000331070B8009326F033954
:101CF0000F0B010F2C6F80EC5FF0336F2C0580EC25
:101D00005FF0335D335F2C6B3233D8B02C272C332C
:101D100032A984EF0EF033512C271200AAEC0FF0F9
:101D2000D8B0120003510719286F6DEC0FF0D8904E
:101D30000751031928AF800F1200286B91EC0FF0A8
:101D4000D8A0A7EC0FF0D8B012007CEC0FF085EC17
:101D50000FF01F0E296FBDEC0FF00B35D8B06DECF6
:101D60000FF0D8A00335D8B01200292FABEF0EF03A
:101D700028B194EC0FF01200286B045105110611E4
:101D800007110008D8A091EC0FF0D8A0A7EC0FF035
:101D9000D8B01200086B096B0A6B0B6BBDEC0FF02F
:101DA0001F0E296FBDEC0FF007510B5DD8A4E5EFB6
:101DB0000EF006510A5DD8A4E5EF0EF00551095D5D
:101DC000D8A4E5EF0EF00451085DD8A0F8EF0EF0AE
:101DD0000451085F0551D8A0053D095F0651D8A000
:101DE000063D0A5F0751D8A0073D0B5FD8900081E0
:101DF000292FD2EF0EF028B194EC0FF0286B91EC64
:101E00000FF0D890C1EC0FF007510B5DD8A415EF7F
:101E10000FF006510A5DD8A415EF0FF00551095DCA
:101E2000D8A415EF0FF00451085DD8A024EF0FF0EF
:101E3000003F24EF0FF0013F24EF0FF0023F24EFAB
:101E40000FF0032BD8B4120028B194EC0FF012005D
:101E50000101286B91EC0FF0D8B01200C6EC0FF026
:101E6000200E296F003701370237033711EE27F0B4
:101E70000A0E2A6FE7360A0EE75CD8B0E76EE55225
:101E80002A2F3AEF0FF0292F32EF0FF028B11D81E2
:101E9000D890120001010A0E286F200E296F11EE52
:101EA0001DF028512A6F0A0ED890E652D8B0E726C6
:101EB000E7322A2F55EF0FF003330233013300339B
:101EC000292F4FEF0FF0E750FF0FD8A00335D8B000
:101ED00012001DB194EC0FF01200045100270551BF
:101EE000D8B0053D01270651D8B0063D022707515D
:101EF000D8B0073D032712000051086F0151096F48
:101F000002510A6F03510B6F12000101006B016B4C
:101F1000026B036B12000101046B056B066B076B10
:101F200012000335D8A012000351800B001F011FBF
:101F3000021F031F003FA4EF0FF0013FA4EF0FF0BB
:101F4000023FA4EF0FF0032B282B032512000735C7
:101F5000D8A012000751800B041F051F061F071F82
:101F6000043FBAEF0FF0053FBAEF0FF0063FBAEFAC
:101F70000FF0072B282B07251200003701370237F7
:101F80000337083709370A370B3712001D6B1E6BF2
:101F90001F6B206B216B226B236B246B256B266BD5
:101FA000276B12001E510F0B1E6F1F510F0B1F6F5F
:101FB00020510F0B206F21510F0B216F22510F0B5E
:101FC000226F23510F0B236F24510F0B246F2551C8
:101FD0000F0B256F26510F0B266F27510F0B276F05
:021FE0001200ED
:10BF0000E844F926000C160C2B0C3F0C520C640C68
:10BF1000760C860C960CA50CB30CC10CCF0CDC0C6B
:06BF2000E80CF40C000C1B
:00000001FF
